
 DaniS506

 Start     Length     Name                   Class
 0001:0000 0003CH     DDHeader               DATA
 0001:003C 00031H     LIBDATA                DATA
 0001:0070 0E496H     _DATA                  DATA
 0001:E506 00000H     CONST                  CONST
 0001:E508 00042H     _BSS                   BSS
 0001:E550 00036H     c_common               BSS
 0002:0000 0000EH     CODE                   CODE
 0002:0010 0022EH     LIBCODE                CODE
 0002:0240 0A808H     _TEXT                  CODE
 0002:AA48 00000H     InitCode               CODE
 0002:AA48 00000H     EndCode                CODE
 0003:0000 008DCH     CSCode                 CODE
 0003:08DC 0008DH     ACPICode               CODE
 0003:096C 0515AH     FCode                  CODE
 0003:5AC8 001E0H     RMCode                 CODE
 0004:0000 0FFFFH     Messages               MSGS

 Origin   Group
 0001:0   DGROUP
 0002:0   STATICGROUP
 0003:0   STATICGROUP2

  Address         Publics by Name

 0003:51BE       @AcceptAEC
 0003:5238       @AcceptAEC2
 0003:4166       @AcceptAHCI
 0003:42B6       @AcceptALI
 0003:3D48       @AcceptAMD
 0003:53CC       @AcceptBCM
 0003:49AE       @AcceptCMD
 0003:4F12       @AcceptCx
 0003:4016       @AcceptGeneric
 0003:504E       @AcceptHPT
 0003:5908       @AcceptInitio
 0003:56DA       @AcceptITE
 0003:38DB       @AcceptITE8213
 0003:537D       @AcceptIXP
 0003:56C9       @AcceptIXPSATA
 0003:57A0       @AcceptJMB
 0003:40BB       @AcceptMarvell
 0003:40A6       @AcceptNetCell
 0003:3E1D       @AcceptNVidia
 0003:5442       @AcceptOPTI
 0003:52C2       @AcceptOSB
 0003:4AB0       @AcceptPDC
 0003:4C17       @AcceptPDCMIO
 0003:4B3E       @AcceptPDCTX2
 0003:3512       @AcceptPIIX
 0003:386E       @AcceptSCH
 0003:5652       @AcceptSII
 0003:45F4       @AcceptSIS
 0003:38AB       @AcceptSMSC
 0003:3924       @AcceptVIA
 0002:7D23       @AcousticEnable
 0003:090B       @ACPIGetPCIIRQs
 0003:08DC       @ACPISetup
 0002:5881       @AddUnit
 0002:6EF0       @AdjustCylinders
 0002:A04E       @AEC2TimingValue
 0002:9F1A       @AECTimingValue
 0002:8DA3       @ALITimingValue
 0003:1BFB       @AllocAdapterResources
 0002:3982       @AllocateUnit
 0003:1B6F       @AllocResource
 0002:7D7D       @APMEnable
 0002:3DF7       @APMResume
 0002:3D88       @APMSuspend
 0003:1D59       @AssignAdapterResources
 0002:584D       @AssignPCIChips
 0002:597F       @AssignSGList
 0002:8A11       @BMCheckIRQ
 0002:7727       @BPBGeometryGet
 0002:0874       @BuildSGList
 0002:8297       @CalculateAdapterTiming
 0002:88D3       @CalculateGenericAdapterTiming
 0003:09AA       @CallAcpiCA
 0003:02E9       @CallCS
 0003:0973       @CallOEMHlp
 0002:3F93       @CardInsertion
 0002:43E6       @CardInsertionDeferred
 0002:3F50       @CardRemoval
 0003:007C       @CardServicesPresent
 0002:1A5C       @CatchInterrupt
 0002:39B4       @ChangeUnitInfo
 0002:30DD       @CheckBusy
 0002:529E       @CheckController
 0003:27ED       @CheckLegacyPorts
 0002:7592       @CheckLVM
 0002:75E1       @CheckMBRConsistency
 0002:30D5       @CheckReady
 0003:2C3B       @CheckSATAPhy
 0003:28AF       @CheckWellknown
 0002:3065       @CheckWorker
 0002:0F66       @ClearIORB
 0002:46D0       @clrmem
 0002:9313       @CMDCheckIRQ
 0002:912D       @CMDTimingValue
 0002:5D08       @CollectPorts
 0003:2CC6       @CollectSCRPorts
 0003:2006       @Command_Parser
 0002:38ED       @CompleteInit
 0002:5ACC       @ConfigureACB
 0002:5D94       @ConfigureController
 0002:5C6D       @ConfigurePCCard
 0003:0DEE       @ConfigurePCI
 0002:5FEE       @ConfigureUnit
 0002:636B       @CountBits
 0002:32D6       @CreateBMSGList
 0003:0108       @CSCardPresent
 0003:03A2       @CSConfigure
 0003:0800       @CSReconfigure
 0003:029A       @CSRegisterClient
 0003:083E       @CSUnconfigure
 0002:9AB6       @CxTimingValue
 0003:1D1E       @DeallocAdapterResources
 0002:399B       @DeallocateUnit
 0002:3C98       @Delay
 0002:6D04       @DetermineUnitGeometry
 0002:051A       @DevHelp_AllocateCtxHook
 0002:0328       @DevHelp_AllocGDTSelector
 0002:055E       @DevHelp_ArmCtxHook
 0002:0346       @DevHelp_AttachDD
 0002:0360       @DevHelp_Beep
 0002:03A6       @DevHelp_CreateInt13VDM
 0002:03F6       @DevHelp_EOI
 0002:0542       @DevHelp_FreeCtxHook
 0002:040C       @DevHelp_GetDOSVar
 0002:05DC       @DevHelp_LockLite
 0002:049C       @DevHelp_PhysToVirt
 0002:04EE       @DevHelp_ProcBlock
 0002:04CC       @DevHelp_ProcRun
 0002:037A       @DevHelp_RegisterDeviceClassLite
 0002:0432       @DevHelp_Save_Message
 0002:03C4       @DevHelp_SetIRQ
 0002:03DE       @DevHelp_UnSetIRQ
 0002:044E       @DevHelp_VerifyAccess
 0002:0588       @DevHelp_VirtToLin
 0002:0470       @DevHelp_VirtToPhys
 0002:05AC       @DevHelp_VMAllocLite
 0002:6206       @DiffTime
 0002:277F       @DoBlockIO
 0002:4D7C       @DoIOCtlPCMCIA
 0002:145B       @DoIOCTLs
 0002:2933       @DoneState
 0002:28B0       @DoOtherIO
 0002:2D3F       @DoReset
 0002:0F8A       @DoSMART
 0002:5486       @DriveInit
 0003:2E6E       @EnumPCIDevices
 0002:3B9D       @Error
 0002:2B43       @ErrorState
 0002:531E       @Execute
 0002:46DD       @fclrmem
 0002:3514       @FillUnitInfo
 0002:4C7E       @FindAdapterForSocket
 0003:1EAD       @FindHotPCCard
 0002:19FD       @FixedInterrupt
 0002:0261       @FixedIRQ0
 0002:0264       @FixedIRQ1
 0002:0267       @FixedIRQ2
 0002:026A       @FixedIRQ3
 0002:026D       @FixedIRQ4
 0002:0270       @FixedIRQ5
 0002:0273       @FixedIRQ6
 0002:0276       @FixedIRQ7
 0002:8D0C       @GenericErrorDMA
 0002:8B8E       @GenericGetTF
 0003:4216       @GenericInitComplete
 0003:4217       @GenericSATA
 0002:8A91       @GenericSetTF
 0002:8CB7       @GenericSetupDMA
 0002:8C74       @GenericStartOp
 0002:8CE5       @GenericStopDMA
 0002:A036       @GetAEC2Pio
 0002:9ECA       @GetAECPio
 0003:4230       @GetAHCISCR
 0002:8D20       @GetALIPio
 0003:2945       @GetBAR
 0002:3101       @GetChangeLine
 0002:65F1       @GetChipPIOMode
 0002:90CC       @GetCMDPio
 0002:9A7E       @GetCxPio
 0002:6498       @GetDeviceDMAMode
 0002:6565       @GetDevicePIOMode
 0002:365F       @GetDeviceTable
 0002:6387       @GetDeviceULTRAMode
 0002:88B1       @GetGenericPio
 0002:9BFF       @GetHPTPio
 0002:1171       @GetInquiryData
 0002:A926       @GetJMBPio
 0002:311C       @GetLockStatus
 0002:8892       @GetNetCellPio
 0002:A29A       @GetOPTIPio
 0002:A0A8       @GetOSBPio
 0003:27D3       @GetPCIBuses
 0002:9390       @GetPDCPio
 0002:82F4       @GetPIIXPio
 0002:39F7       @GetQueueStatus
 0003:0AC7       @GetRegB
 0003:0B11       @GetRegD
 0003:0AED       @GetRegW
 0002:8373       @GetSCHPio
 0002:A48A       @GetSIIPio
 0002:A4B1       @GetSIISATAPio
 0002:8F0E       @GetSISPio
 0002:1024       @GetSmartStatus
 0002:3A08       @GetUnitResources
 0002:3136       @GetUnitStatus
 0002:8658       @GetVIAPio
 0003:3251       @HandleFoundAdapter
 0002:0278       @HandleInterrupts
 0002:53BE       @HookIRQ
 0002:9E8D       @HPT36xErrorDMA
 0002:9E08       @HPT36xPreReset
 0002:9E30       @HPT36xSetupDMA
 0002:9EA9       @HPT37xErrorDMA
 0002:9E13       @HPT37xPreReset
 0002:9E5A       @HPT37xSetupDMA
 0002:9D8A       @HPTCheckIRQ
 0002:9BB2       @HPTClkIdx
 0002:9DF9       @HPTEnableInt
 0002:9C3D       @HPTTimingValue
 0002:7249       @IDEGeomExtract
 0002:6674       @IdentifyDevice
 0002:6F69       @IdentifyGeometryGet
 0002:7C9A       @IdleTimerEnable
 0002:7B34       @IDStringsExtract
 0002:0A5D       @InB
 0002:0A5D       @InB2
 0002:0A8E       @InBd
 0002:0A89       @InBdms
 0002:0AD1       @InD
 0002:0AD1       @InD2
 0002:0B29       @InDd
 0002:0B24       @InDdms
 0002:1C1D       @InitACBRequest
 0002:20A5       @InitBlockIO
 0002:A9B6       @InitioCheckIRQ
 0002:A9B5       @InitioErrorDMA
 0002:A948       @InitioSetupDMA
 0002:A95C       @InitioStartOp
 0002:A995       @InitioStopDMA
 0002:3CEC       @InitUnitSync
 0003:349A       @Int13DoRequest
 0003:343D       @Int13Fun08GetLogicalGeom
 0002:74CC       @Int13GeometryGet
 0002:25F0       @InterruptState
 0002:0A99       @InW
 0002:0A99       @InW2
 0002:0ACA       @InWd
 0002:0AC5       @InWdms
 0002:10C1       @IOCtlRead
 0002:46BA       @IODly
 0002:46C5       @IODlyFar
 0002:3BAD       @IORBDone
 0002:0EF2       @IssueCommand
 0002:0F46       @IssueCommandTO
 0002:1348       @IssueGetPowerStatus
 0002:1200       @IssueOneByte
 0002:4019       @IssueSATAReset
 0002:1318       @IssueSetFeatures
 0002:1368       @IssueSetIdle
 0002:1226       @IssueSetMax
 0002:A854       @ITETimingValue
 0003:1F96       @LocateATEntry
 0002:7394       @LogGeomCalculate
 0002:7400       @LogGeomCalculateLBAAssist
 0002:7D9C       @LPMEnable
 0002:3168       @MapError
 0002:32AD       @MapMediaStatus
 0002:139D       @MapUnit
 0002:7B71       @MediaStatusEnable
 0002:7BF6       @MultipleModeEnable
 0003:2D20       @nextController
 0002:33BA       @NextIORB
 0002:585E       @NoMaster
 0002:895D       @NonsharedCheckIRQ
 0002:5379       @NoOp
 0002:3BE2       @NotifyFLT
 0002:A2D1       @OPTITimingValue
 0002:A0D4       @OSBTimingValue
 0002:0968       @OutB
 0002:0968       @OutB2
 0002:09A1       @OutBd
 0002:0994       @OutBdms
 0002:09E1       @OutD
 0002:09E1       @OutD2
 0002:09B5       @OutW
 0002:09B5       @OutW2
 0003:10DB       @ParseCmdLine
 0003:0A38       @PciGetReg
 0003:09E6       @PciSetReg
 0003:004A       @PCMCIASetup
 0002:981E       @PDCPostReset
 0002:9841       @PDCPreReset
 0002:9856       @PDCSetupDMA
 0002:98A6       @PDCStartOp
 0002:93CE       @PDCTimingValue
 0002:7B17       @PhysGeomValidate
 0002:8232       @PickClockIndex
 0002:8398       @PIIXTimingValue
 0003:1501       @PortToPhys
 0002:4845       @PreProcessIORBs
 0003:155A       @PrintAdapterInfo
 0003:16BD       @PrintInfo
 0002:683A       @prntf
 0003:2A46       @ProbeChannel
 0003:1ABB       @ProcessVerboseTimings
 0002:A08F       @ProgramAEC2Chip
 0002:9F8D       @ProgramAECChip
 0002:8E47       @ProgramALIChip
 0002:91D3       @ProgramCMDChip
 0002:9B4D       @ProgramCxChip
 0002:9CD7       @ProgramHPTChip
 0002:A8D1       @ProgramITEChip
 0002:A373       @ProgramOPTIChip
 0002:A163       @ProgramOSBChip
 0002:9562       @ProgramPDCChip
 0002:96A2       @ProgramPDCChipTX2
 0002:94B3       @ProgramPDCIO
 0002:843B       @ProgramPIIXChip
 0002:85DA       @ProgramSCH
 0002:A59C       @ProgramSIIChip
 0002:A618       @ProgramSIISATAChip
 0002:9092       @ProgramSIS2Chip
 0002:904B       @ProgramSISChip
 0002:874E       @ProgramVIAChip
 0002:9749       @PromiseCheckIRQ
 0003:4B9D       @PromiseInitComplete
 0002:99D5       @PromiseMCheckIRQ
 0002:99D4       @PromiseMErrorDMA
 0002:990F       @PromiseMSetupDMA
 0002:9923       @PromiseMStartOp
 0002:99A1       @PromiseMStopDMA
 0002:96B9       @PromiseTX2CheckIRQ
 0002:49E6       @RConfigB
 0002:49F4       @RConfigW
 0002:7AC6       @ReadAndExtractBPB
 0002:4970       @ReadConfigB
 0002:49BD       @ReadConfigD
 0002:4998       @ReadConfigW
 0002:608E       @ReadDrive
 0002:A268       @ReadIDEReg
 0003:0B39       @ReadPCIConfigSpace
 0002:3EE5       @ReConfigureUnit
 0002:6271       @RegisterADD
 0002:545C       @RehookIRQ
 0002:3D55       @ReInitUnit
 0002:2DDF       @ResetCheck
 0002:481A       @ResumeIORBReq
 0002:1BE4       @RetryState
 0002:024C       @safeCLR32
 0002:0253       @safeDEC
 0002:0243       @safeGET32
 0002:025A       @safeINC
 0002:0240       @safeXCHG
 0002:40ED       @SATARemoval
 0003:1A1D       @SaveMsg
 0003:0FCE       @ScanForOtherADDs
 0002:58C0       @ScanForUnits
 0002:30E5       @SelectUnit
 0002:2F7C       @SendCmdPacket
 0002:2470       @SetIOAddress
 0003:2859       @SetLatency
 0002:3100       @SetMediaGeometry
 0003:1091       @SetOption
 0003:0A94       @SetRegB
 0003:0AB4       @SetRegD
 0003:0AAA       @SetRegW
 0002:2C9A       @SetRetryState
 0002:8D54       @SetupALI
 0002:81F6       @SetupCommon
 0002:80A4       @SetupCommonPost
 0002:7E0E       @SetupCommonPre
 0002:1EB5       @SetupFromATA
 0003:4F26       @SetupHPTPLL
 0002:2025       @SetupIdentify
 0003:274C       @SetupOEMHlp
 0002:580D       @SetupPCI
 0002:57C5       @SetupPCMCIA
 0002:93AF       @SetupPDCTX2
 0003:2B96       @SetupT13StandardController
 0002:A79D       @SIICheckIRQ
 0003:5488       @SiISATA
 0002:A654       @SIISetTF
 0002:A689       @SIIStartOp
 0002:A71A       @SIIStartStop
 0002:A4EE       @SIITimingValue
 0002:8FEA       @SIS2TimingValue
 0002:8F5A       @SISTimingValue
 0002:23C0       @StartBlockIO
 0002:3FAF       @StartDetect
 0002:4129       @StartDetectSATA
 0002:1B84       @StartIO
 0002:2125       @StartOtherIO
 0002:1970       @StartSM
 0002:1A87       @StartState
 0002:46F1       @strnswap
 0002:47F2       @Suspend
 0002:476A       @SuspendIORBReq
 0002:4813       @SuspendState
 0002:4FEF       @TestChannel
 0002:4EC2       @TestStatus50us
 0002:6223       @TotalTime
 0002:6156       @TraceCh
 0002:6194       @TraceTime
 0002:61C6       @TraceTTime
 0002:4F98       @TryCommand
 0003:0382       @TryIO
 0003:0345       @TryIRQ
 0003:1A85       @TTYWrite
 0002:6240       @TWrite
 0002:6289       @UCBSetupDMAPIO
 0002:543B       @UnhookIRQ
 0002:3D72       @UnitFlush
 0002:701A       @UnlockMax
 0003:339A       @VDMInt13Create
 0002:5A17       @VerifyInitPost
 0002:8692       @VIATimingValue
 0002:2FEF       @WaitDRQ
 0002:4EF8       @WaitNotBusy
 0002:4F4B       @WaitNotBusyDRQ
 0002:4A5D       @WConfigB
 0002:4A51       @WConfigBI
 0002:4A77       @WConfigD
 0002:4A6B       @WConfigW
 0002:4A00       @WriteConfigB
 0002:4A1B       @WriteConfigBI
 0002:4A3D       @WriteConfigD
 0002:4A32       @WriteConfigW
 0003:0C99       @WritePCIConfigSpace
 0002:4738       @_strncmp
 0002:6CA6       @_strncpy
 0002:011C       ADD_CancelTimer
 0002:0095       ADD_DeInstallTimer
 0002:0010       ADD_InitTimer
 0002:00A9       ADD_StartTimerMS
 0002:05F4       ADD_XFERIO
 0000:0000  Imp  DOS32FLATDS          (DOSCALLS.370)
 0000:0000  Imp  DOSIODELAYCNT        (DOSCALLS.427)
 0002:013F       f_ADD_TimerHandler
 0003:5AD0       MY_DEVHELP_ATTACHDD
 0001:02C2       _ACBPtrs
 0001:1C1C       _ACPICA_DDName
 0001:1C3E       _ACPIIDC
 0001:DDBC       _AdaptDescriptNameTxt
 0001:03F4       _AdapterNameATAPI
 0001:0406       _AdapterNamePCCrd
 0001:DDD2       _AdapterStruct
 0001:2974       _AdapterTable
 0002:330C       _ADDEntryPoint
 0001:036A       _ADDHandle
 0001:D7CA       _AdptMsgs
 0001:05C4       _AEC62X0_ModeSets
 0001:D85E       _AEC62xMsgtxt
 0001:D82A       _ALI5229Msgtxt
 0001:0430       _ALI_ModeSets
 0001:0450       _ALI_Ultra100ModeSets
 0001:043C       _ALI_UltraModeSets
 0001:D856       _AMDxMsgtxt
 0002:0190       _APMAttach
 0002:022B       _APMDeregister
 0002:3CAF       _APMEventHandler
 0002:01BE       _APMRegister
 0001:D7F8       _ATAPIMsg
 0001:D7B5       _ATAPISlaveChk
 0001:1C52       _BasePortpref
 0001:039C       _Beeps
 0001:0374       _BIOSActive
 0001:0375       _BIOSInt13
 0001:8B34       _BootRecord
 0001:0D46       _BroadcomMsgtxt
 0001:036D       _cAdapters
 0002:4B5D       _CalculateLoss
 0003:0000       _CallCardServices
 0003:5C72       _CallRM
 0001:DA78       _cc
 0001:036C       _cChips
 0001:0806       _CfgAEC
 0001:0774       _CfgALI
 0001:07CE       _CfgCMD
 0001:07E6       _CfgCX
 0001:0756       _CfgGeneric
 0001:07A4       _CfgHPT36x
 0001:07A0       _CfgHPT37x
 0001:074C       _CfgICH
 0001:0854       _CfgITE
 0001:0824       _CfgNFC
 0001:075E       _CfgNull
 0001:0816       _CfgOPTI
 0001:0800       _CfgOSB
 0001:0788       _CfgPDC
 0001:0754       _CfgPIIX
 0001:0752       _CfgPIIX3
 0001:074E       _CfgPIIX4
 0001:0836       _CfgSII
 0001:07A8       _CfgSIS
 0001:07B8       _CfgSIS2
 0001:0760       _CfgVIA
 0001:1CB4       _ChipTable
 0001:1C5A       _CIInfo
 0001:0AE6       _CListCAEC
 0001:0A06       _CListCALi
 0001:0B06       _CListCBCMSata
 0001:0CF2       _CListCInitio
 0001:0868       _CListCIntel
 0001:0C70       _CListCIXP
 0001:0C96       _CListCIXPA
 0001:0C88       _CListCIXPS
 0001:0CCE       _CListCMarvell
 0001:0B22       _CListCNvidia
 0001:0B10       _CListCOpti
 0001:0A4A       _CListCPromise
 0001:0A78       _CListCPromiseS
 0001:0A5C       _CListCPromiseTX
 0001:0C54       _CListCSiI
 0001:0A18       _CListCSiS
 0001:09BE       _CListCVia
 0001:0AEC       _CListFAEC
 0001:0AF4       _CListFAEC2
 0001:0A0C       _CListFALi
 0001:0AD8       _CListFAMD
 0001:0B0C       _CListFBCMSata
 0001:0A3E       _CListFCMD
 0001:0AC6       _CListFCyrix
 0001:0ACA       _CListFHighPoint
 0001:098E       _CListFIntel
 0001:09BA       _CListFiSCH
 0001:0C66       _CListFITE
 0001:0C6C       _CListFITE2
 0001:0C82       _CListFIXP
 0001:0CB4       _CListFIXPA
 0001:0C92       _CListFIXPS
 0001:0C50       _CListFNatSemi
 0001:0C38       _CListFNvidia
 0001:0B1A       _CListFOpti
 0001:0A54       _CListFPromise
 0001:0AB6       _CListFPromiseS
 0001:0A72       _CListFPromiseTX
 0001:0AFC       _CListFServerWorks
 0001:0C5E       _CListFSiI
 0001:0A2E       _CListFSiS
 0001:0AF8       _CListFSMSC
 0001:09F4       _CListFVia
 0001:0CB8       _CListFVSB
 0001:0CF8       _CListInitio
 0001:0CC0       _CListJMicron
 0001:0CEC       _CListMarvell
 0001:0CBC       _CListNetCell
 0001:0866       _CListNULL
 0001:D804       _CMD64xMsgtxt
 0001:0418       _CmdTable
 0001:0458       _CMD_ModeSets
 0001:0464       _CMD_UltraModeSets
 0001:E154       _counted
 0002:4CB3       _CSCallbackHandler
 0002:4504       _CSCallbackStub
 0001:1C54       _CSCtxHook
 0001:1C4A       _CSHandle
 0002:02A0       _CSHookHandler
 0001:1C32       _CSIDC
 0001:1C58       _CSIrqAvail
 0001:036F       _cSockets
 0001:1C4C       _CSRegistrationComplete
 0002:000A       _CSSel
 0001:036E       _cUnits
 0001:03A6       _CurLevel
 0001:03A4       _CurPCIInfo
 0001:0CFC       _Cx5530Msgtxt
 0001:04AC       _CX_DMAModeSets
 0001:047C       _CX_PIOModeSets
 0001:038E       _Debug
 0001:0070       _Delay500
 0002:461D       _DelayedReset
 0002:45FD       _DelayedRetry
 0001:DDEA       _DevDescriptNameTxt
 0001:0352       _Device_Help
 0001:DDFA       _DevStruct
 0001:0000       _DiskDDHeader
 0001:0370       _DriveId
 0001:DDA0       _DriverStruct
 0001:DD74       _DrvrDescriptTxt
 0001:DD72       _DrvrNameSize
 0001:DD64       _DrvrNameTxt
 0002:0008       _DSSel
 0001:8FCA       _DTMem
 0002:4638       _ElapsedTimer
 0001:0386       _ElapsedTimerHandle
 0001:0376       _EzDrivePresent
 0001:1C4F       _FirstSocket
 0001:03A2       _Fixes
 0002:000C       _FlatSel
 0001:E564       _fs
 0001:D7BA       _GenericBM
 0001:0D60       _GenericMsgtxt
 0003:5C9A       _GetCS
 0001:03AE       _GetTuple
 0001:0366       _hDriver
 0001:D84E       _HPT36xMsgtxt
 0001:0532       _HPT37x_ModeSets
 0001:0556       _HPT37x_UltraModeSets
 0001:04FC       _HPT_ModeSets
 0001:0520       _HPT_UltraModeSets
 0001:D842       _ICHxMsgtxt
 0001:D8C6       _IDERMsgtxt
 0002:4667       _IdleTicker
 0001:0388       _IdleTickerHandle
 0001:0322       _IHdr
 0001:0371       _InitActive
 0001:0373       _InitComplete
 0001:0372       _InitIOComplete
 0001:D8B6       _InitioMsgtxt
 0001:8F70       _InitIORB
 0001:D7C2       _InitMsg
 0002:4171       _InsertHandler
 0001:1C50       _Inserting
 0001:8F52       _IOCtlACPI
 0001:8F34       _IOCtlRP
 0001:0384       _IODelayCount
 0001:1C51       _IRQprefLevel
 0002:451E       _IRQTimer
 0001:D886       _ITEMsgtxt
 0001:0738       _ITE_ModeSets
 0001:073E       _ITE_UltraModeSets
 0001:0D3E       _IXPMsgtxt
 0001:D88E       _JMMsgtxt
 0001:03AA       _LastAccessedPCCardUnit
 0001:03A8       _LastAccessedUnit
 0001:D96E       _length
 0001:039D       _LinesPrinted
 0002:02BC       _LoadFlatGS
 0001:D8AA       _MarvellMsgtxt
 0001:1C4E       _MaxNumSockets
 0001:E576       _MemTop
 0002:4B80       _MPIfIOCtl
 0001:D7EE       _MsgAML
 0001:D7F4       _MsgBMOn
 0004:0000       _MsgBuffer
 0004:FFFF       _MsgBufferEnd
 0001:D7F2       _MsgEzDriveFBP
 0001:D7EC       _MsgLBAon
 0001:D7FA       _MsgNull
 0001:D7F0       _MsgONTrackOn
 0001:D7EA       _MsgSMS
 0001:D7F6       _MsgTypeMDMAOn
 0001:037C       _msTimer
 0001:0D2C       _NetCellMsgtxt
 0001:D876       _NForceMsgtxt
 0002:4E9C       _NotifyIORBDone
 0001:03A0       _NotShutdown
 0001:D3CA       _npTrace
 0001:0D1C       _NsSCxMsgtxt
 0001:1C4D       _NumSockets
 0001:1C26       _OemHlpIDC
 0001:1C08       _OEMHLP_DDName
 0001:0D12       _OPTIMsgtxt
 0001:072C       _OPTI_ModeSets
 0001:DD02       _opttable
 0001:DBD2       _OPT_80WIRE
 0001:DBDA       _OPT_ADAPTER
 0001:DBE2       _OPT_APM
 0001:DBEA       _OPT_BAY
 0001:DBF2       _OPT_BM_DMA
 0001:DBFA       _OPT_DEBUG
 0001:DC02       _OPT_DM
 0001:DCFA       _OPT_END
 0001:DC0A       _OPT_FIXES
 0001:DC12       _OPT_FORCEGBM
 0001:DC1A       _OPT_GBM
 0001:DC2A       _OPT_IDLETIMER
 0001:DC32       _OPT_IGNORE
 0001:DC22       _OPT_IRQ
 0001:DCA2       _OPT_IRQTIMEOUT
 0001:DC3A       _OPT_LATENCY
 0001:DC42       _OPT_LOC
 0001:DC4A       _OPT_LPM
 0001:DC52       _OPT_MAXRATE
 0001:DC5A       _OPT_NOISE
 0001:DBB2       _OPT_NOSHTDWN
 0001:DB82       _OPT_NOTBEEP
 0001:DBA2       _OPT_NOTREMOVABLE
 0001:DB8A       _OPT_NOT_BIOS
 0001:DB92       _OPT_NOT_BM_DMA
 0001:DB9A       _OPT_NOT_DM
 0001:DBAA       _OPT_NOT_SETMAX
 0001:DBBA       _OPT_NOT_SMS
 0001:DBC2       _OPT_NOT_VERBOSE
 0001:DBCA       _OPT_NOT_VPAUSE
 0001:DC82       _OPT_P
 0001:DC6A       _OPT_PCICLOCK
 0001:DC62       _OPT_PCMCIA
 0001:DC7A       _OPT_PF
 0001:DC72       _OPT_PORT
 0001:DC8A       _OPT_REMOVABLE
 0001:DC92       _OPT_SHTDWN
 0001:DC9A       _OPT_SMS
 0001:DCAA       _OPT_T
 0001:DCBA       _OPT_U
 0001:DCB2       _OPT_UNIT
 0001:DCC2       _OPT_VERBOSE
 0001:DCD2       _OPT_VERBOSEL
 0001:DCE2       _OPT_VERBOSELL
 0001:DCCA       _OPT_VPAUSE
 0001:DCDA       _OPT_VPAUSEL
 0001:DCEA       _OPT_VPAUSELL
 0001:DCF2       _OPT_WP
 0001:D864       _OSBMsgtxt
 0001:0704       _OSB_ModeSets
 0001:0710       _OSB_UltraModeSets
 0001:DA7C       _outbuf
 0001:DB7C       _outbuf_len
 0001:D8D6       _ParmErrMsg
 0001:8D34       _PartitionBootRecord
 0001:0302       _PCCardPtrs
 0001:038B       _PCIClock
 0001:038C       _PCIClockIndex
 0001:0D68       _PCIDevice
 0001:D7C1       _PCILatency
 0001:038A       _PCInumBuses
 0001:1C12       _PCMCIA_DDName
 0001:D95E       _pcmdline1
 0001:D962       _pcmdline_slash
 0001:D966       _pcmdline_start
 0001:D832       _PDCxMsgtxt
 0001:0572       _PDC_100ModeSets
 0001:0578       _PDC_133ModeSets
 0001:0598       _PDC_DMA100ModeSets
 0001:05A8       _PDC_DMA133ModeSets
 0001:0588       _PDC_DMA66ModeSets
 0001:057E       _PDC_DMAModeSets
 0001:056C       _PDC_ModeSets
 0001:D7B6       _pDDD_Parm_List
 0001:0380       _pDriverTable
 0001:DA70       _pend_option
 0001:0378       _pGlobal
 0001:D80C       _PIIXxMsgtxt
 0001:05C8       _PIIX_ModeSets
 0001:05D4       _PIIX_UltraModeSets
 0001:DB7E       _poutbuf
 0001:DA74       _poutbuf1
 0001:DA76       _poutbuf_end
 0001:03A1       _PowerState
 0001:0362       _ppDataSeg
 0001:D89C       _PromiseMIOtxt
 0001:DA72       _ptable_option
 0001:14D0       _Queue
 0001:0398       _ReadPtr
 0001:E578       _Register
 0001:03A7       _RegOffset
 0001:18D4       _ReqCount
 0003:5C0C       _RMAllocResource
 0003:5B98       _RMCreateAdapter
 0003:5BD2       _RMCreateDevice
 0003:5AF2       _RMCreateDriver
 0003:5C46       _RMDeallocResource
 0003:5B6C       _RMDestroyDriver
 0001:035E       _RMFlags
 0001:E4FA       _RMIDCTable
 0001:0356       _RM_Help0
 0001:035A       _RM_Help3
 0002:0B32       _S506Str1
 0001:E550       _sbuf
 0001:0D4C       _SCHMsgtxt
 0001:14D4       _ScratchBuf
 0001:14C8       _ScratchSGList
 0001:D7FC       _SII68xMsgtxt
 0001:05C0       _SII_MDMAModeSets
 0001:05BA       _SII_ModeSets
 0001:0662       _SIS2_100ModeSets
 0001:066E       _SIS2_133ModeSets
 0001:067A       _SIS2_UltraModeSets
 0001:D822       _SiS5513Msgtxt
 0001:060C       _SIS_ModeSets
 0001:0654       _SIS_Ultra100ModeSets
 0001:065A       _SIS_Ultra133ModeSets
 0001:063C       _SIS_Ultra66ModeSets
 0001:0624       _SIS_UltraModeSets
 0001:0D08       _SLC90E66Msgtxt
 0001:05F0       _SMSC_UltraModeSets
 0001:02E2       _SocketPtrs
 0002:6826       _sprntf
 0001:D96C       _state_index
 0003:096C       _StubVDMInt13CallBack
 0001:18D6       _TimerPool
 0001:D970       _tokvbuf
 0001:D96A       _tokv_index
 0001:D3CC       _TraceBuffer
 0001:039F       _TraceErrors
 0001:039E       _TracerEnabled
 0002:6168       _TraceStr
 0001:D7DE       _UnitMsgs
 0001:03AC       _UStatus
 0001:E086       _VBlankLine
 0001:DF9C       _VBPBInfo
 0001:DF14       _VControllerInfo
 0001:E10E       _VDMAString
 0001:DEBE       _VDMDskBlkID
 0001:DE0A       _VDMInt13
 0001:DE08       _VDMInt13Active
 0001:DEC2       _VDMInt13BlkID
 0003:34DC       _VDMInt13CallBack
 0001:DE06       _VDMInt13Created
 0001:DD9A       _VendorNameTxt
 0001:D7B4       _Verbose
 0001:D91A       _VersionMsg
 0001:DFB2       _VGeomInfo0
 0001:DFF2       _VGeomInfo1
 0001:E022       _VGeomInfo2
 0001:E050       _VGeomInfo3
 0001:DFA2       _VI13Info
 0001:D81A       _VIA571Msgtxt
 0001:0D56       _VIASBMsgtxt
 0001:0688       _VIA_ModeSets
 0001:06CC       _VIA_Ultra100ModeSets
 0001:06E8       _VIA_Ultra133ModeSets
 0001:06B0       _VIA_Ultra66ModeSets
 0001:0694       _VIA_UltraModeSets
 0001:DFA8       _VIDEInfo
 0001:DF84       _VModelInfo
 0001:DF90       _VModelUnknown
 0001:E088       _VPauseVerbose0
 0001:E0B0       _VPauseVerbose1
 0001:DEFE       _VPCardInfo
 0001:DEC6       _VPCIInfo
 0001:E120       _VPIOString
 0001:E0DA       _VSata0
 0001:E0E4       _VSata1
 0001:E0F0       _VSata2
 0001:E0D6       _VString
 0001:E0FC       _VULTRADMAString
 0001:DF46       _VUnitInfo1
 0001:DF62       _VUnitInfo2
 0001:0390       _WritePtr
 0001:0396       _WritePtrErr
 0001:0394       _WritePtrRestart
 0001:D7BE       _xBridgeDevice
 0001:D7BC       _xBridgePCIAddr
 0001:D7C0       _xBridgeRevision
 0002:4AE9       __aFlmul
 0002:4A9B       __aFlshl
 0002:4B14       __aFuldiv
 0002:4AE9       __aFulmul
 0002:4B44       __aFulrem
 0002:4AB1       __aFulshr
 0002:4E50       __aNFauldiv
 0002:4E76       __aNFaulrem
 0002:4E32       __aNFaulshr
 0002:4ABC       __aNlmul
 0002:4A90       __aNlshl
 0002:4AD0       __aNNalmul
 0002:4AD0       __aNNaulmul
 0002:4AFD       __aNuldiv
 0002:4ABC       __aNulmul
 0002:4B2B       __aNulrem
 0002:4AA6       __aNulshr
 0002:AA48       __CodeEnd

  Address         Publics by Value

 0000:0000  Imp  DOSIODELAYCNT        (DOSCALLS.427)
 0000:0000  Imp  DOS32FLATDS          (DOSCALLS.370)
 0001:0000       _DiskDDHeader
 0001:0070       _Delay500
 0001:02C2       _ACBPtrs
 0001:02E2       _SocketPtrs
 0001:0302       _PCCardPtrs
 0001:0322       _IHdr
 0001:0352       _Device_Help
 0001:0356       _RM_Help0
 0001:035A       _RM_Help3
 0001:035E       _RMFlags
 0001:0362       _ppDataSeg
 0001:0366       _hDriver
 0001:036A       _ADDHandle
 0001:036C       _cChips
 0001:036D       _cAdapters
 0001:036E       _cUnits
 0001:036F       _cSockets
 0001:0370       _DriveId
 0001:0371       _InitActive
 0001:0372       _InitIOComplete
 0001:0373       _InitComplete
 0001:0374       _BIOSActive
 0001:0375       _BIOSInt13
 0001:0376       _EzDrivePresent
 0001:0378       _pGlobal
 0001:037C       _msTimer
 0001:0380       _pDriverTable
 0001:0384       _IODelayCount
 0001:0386       _ElapsedTimerHandle
 0001:0388       _IdleTickerHandle
 0001:038A       _PCInumBuses
 0001:038B       _PCIClock
 0001:038C       _PCIClockIndex
 0001:038E       _Debug
 0001:0390       _WritePtr
 0001:0394       _WritePtrRestart
 0001:0396       _WritePtrErr
 0001:0398       _ReadPtr
 0001:039C       _Beeps
 0001:039D       _LinesPrinted
 0001:039E       _TracerEnabled
 0001:039F       _TraceErrors
 0001:03A0       _NotShutdown
 0001:03A1       _PowerState
 0001:03A2       _Fixes
 0001:03A4       _CurPCIInfo
 0001:03A6       _CurLevel
 0001:03A7       _RegOffset
 0001:03A8       _LastAccessedUnit
 0001:03AA       _LastAccessedPCCardUnit
 0001:03AC       _UStatus
 0001:03AE       _GetTuple
 0001:03F4       _AdapterNameATAPI
 0001:0406       _AdapterNamePCCrd
 0001:0418       _CmdTable
 0001:0430       _ALI_ModeSets
 0001:043C       _ALI_UltraModeSets
 0001:0450       _ALI_Ultra100ModeSets
 0001:0458       _CMD_ModeSets
 0001:0464       _CMD_UltraModeSets
 0001:047C       _CX_PIOModeSets
 0001:04AC       _CX_DMAModeSets
 0001:04FC       _HPT_ModeSets
 0001:0520       _HPT_UltraModeSets
 0001:0532       _HPT37x_ModeSets
 0001:0556       _HPT37x_UltraModeSets
 0001:056C       _PDC_ModeSets
 0001:0572       _PDC_100ModeSets
 0001:0578       _PDC_133ModeSets
 0001:057E       _PDC_DMAModeSets
 0001:0588       _PDC_DMA66ModeSets
 0001:0598       _PDC_DMA100ModeSets
 0001:05A8       _PDC_DMA133ModeSets
 0001:05BA       _SII_ModeSets
 0001:05C0       _SII_MDMAModeSets
 0001:05C4       _AEC62X0_ModeSets
 0001:05C8       _PIIX_ModeSets
 0001:05D4       _PIIX_UltraModeSets
 0001:05F0       _SMSC_UltraModeSets
 0001:060C       _SIS_ModeSets
 0001:0624       _SIS_UltraModeSets
 0001:063C       _SIS_Ultra66ModeSets
 0001:0654       _SIS_Ultra100ModeSets
 0001:065A       _SIS_Ultra133ModeSets
 0001:0662       _SIS2_100ModeSets
 0001:066E       _SIS2_133ModeSets
 0001:067A       _SIS2_UltraModeSets
 0001:0688       _VIA_ModeSets
 0001:0694       _VIA_UltraModeSets
 0001:06B0       _VIA_Ultra66ModeSets
 0001:06CC       _VIA_Ultra100ModeSets
 0001:06E8       _VIA_Ultra133ModeSets
 0001:0704       _OSB_ModeSets
 0001:0710       _OSB_UltraModeSets
 0001:072C       _OPTI_ModeSets
 0001:0738       _ITE_ModeSets
 0001:073E       _ITE_UltraModeSets
 0001:074C       _CfgICH
 0001:074E       _CfgPIIX4
 0001:0752       _CfgPIIX3
 0001:0754       _CfgPIIX
 0001:0756       _CfgGeneric
 0001:075E       _CfgNull
 0001:0760       _CfgVIA
 0001:0774       _CfgALI
 0001:0788       _CfgPDC
 0001:07A0       _CfgHPT37x
 0001:07A4       _CfgHPT36x
 0001:07A8       _CfgSIS
 0001:07B8       _CfgSIS2
 0001:07CE       _CfgCMD
 0001:07E6       _CfgCX
 0001:0800       _CfgOSB
 0001:0806       _CfgAEC
 0001:0816       _CfgOPTI
 0001:0824       _CfgNFC
 0001:0836       _CfgSII
 0001:0854       _CfgITE
 0001:0866       _CListNULL
 0001:0868       _CListCIntel
 0001:098E       _CListFIntel
 0001:09BA       _CListFiSCH
 0001:09BE       _CListCVia
 0001:09F4       _CListFVia
 0001:0A06       _CListCALi
 0001:0A0C       _CListFALi
 0001:0A18       _CListCSiS
 0001:0A2E       _CListFSiS
 0001:0A3E       _CListFCMD
 0001:0A4A       _CListCPromise
 0001:0A54       _CListFPromise
 0001:0A5C       _CListCPromiseTX
 0001:0A72       _CListFPromiseTX
 0001:0A78       _CListCPromiseS
 0001:0AB6       _CListFPromiseS
 0001:0AC6       _CListFCyrix
 0001:0ACA       _CListFHighPoint
 0001:0AD8       _CListFAMD
 0001:0AE6       _CListCAEC
 0001:0AEC       _CListFAEC
 0001:0AF4       _CListFAEC2
 0001:0AF8       _CListFSMSC
 0001:0AFC       _CListFServerWorks
 0001:0B06       _CListCBCMSata
 0001:0B0C       _CListFBCMSata
 0001:0B10       _CListCOpti
 0001:0B1A       _CListFOpti
 0001:0B22       _CListCNvidia
 0001:0C38       _CListFNvidia
 0001:0C50       _CListFNatSemi
 0001:0C54       _CListCSiI
 0001:0C5E       _CListFSiI
 0001:0C66       _CListFITE
 0001:0C6C       _CListFITE2
 0001:0C70       _CListCIXP
 0001:0C82       _CListFIXP
 0001:0C88       _CListCIXPS
 0001:0C92       _CListFIXPS
 0001:0C96       _CListCIXPA
 0001:0CB4       _CListFIXPA
 0001:0CB8       _CListFVSB
 0001:0CBC       _CListNetCell
 0001:0CC0       _CListJMicron
 0001:0CCE       _CListCMarvell
 0001:0CEC       _CListMarvell
 0001:0CF2       _CListCInitio
 0001:0CF8       _CListInitio
 0001:0CFC       _Cx5530Msgtxt
 0001:0D08       _SLC90E66Msgtxt
 0001:0D12       _OPTIMsgtxt
 0001:0D1C       _NsSCxMsgtxt
 0001:0D2C       _NetCellMsgtxt
 0001:0D3E       _IXPMsgtxt
 0001:0D46       _BroadcomMsgtxt
 0001:0D4C       _SCHMsgtxt
 0001:0D56       _VIASBMsgtxt
 0001:0D60       _GenericMsgtxt
 0001:0D68       _PCIDevice
 0001:14C8       _ScratchSGList
 0001:14D0       _Queue
 0001:14D4       _ScratchBuf
 0001:18D4       _ReqCount
 0001:18D6       _TimerPool
 0001:1C08       _OEMHLP_DDName
 0001:1C12       _PCMCIA_DDName
 0001:1C1C       _ACPICA_DDName
 0001:1C26       _OemHlpIDC
 0001:1C32       _CSIDC
 0001:1C3E       _ACPIIDC
 0001:1C4A       _CSHandle
 0001:1C4C       _CSRegistrationComplete
 0001:1C4D       _NumSockets
 0001:1C4E       _MaxNumSockets
 0001:1C4F       _FirstSocket
 0001:1C50       _Inserting
 0001:1C51       _IRQprefLevel
 0001:1C52       _BasePortpref
 0001:1C54       _CSCtxHook
 0001:1C58       _CSIrqAvail
 0001:1C5A       _CIInfo
 0001:1CB4       _ChipTable
 0001:2974       _AdapterTable
 0001:8B34       _BootRecord
 0001:8D34       _PartitionBootRecord
 0001:8F34       _IOCtlRP
 0001:8F52       _IOCtlACPI
 0001:8F70       _InitIORB
 0001:8FCA       _DTMem
 0001:D3CA       _npTrace
 0001:D3CC       _TraceBuffer
 0001:D7B4       _Verbose
 0001:D7B5       _ATAPISlaveChk
 0001:D7B6       _pDDD_Parm_List
 0001:D7BA       _GenericBM
 0001:D7BC       _xBridgePCIAddr
 0001:D7BE       _xBridgeDevice
 0001:D7C0       _xBridgeRevision
 0001:D7C1       _PCILatency
 0001:D7C2       _InitMsg
 0001:D7CA       _AdptMsgs
 0001:D7DE       _UnitMsgs
 0001:D7EA       _MsgSMS
 0001:D7EC       _MsgLBAon
 0001:D7EE       _MsgAML
 0001:D7F0       _MsgONTrackOn
 0001:D7F2       _MsgEzDriveFBP
 0001:D7F4       _MsgBMOn
 0001:D7F6       _MsgTypeMDMAOn
 0001:D7F8       _ATAPIMsg
 0001:D7FA       _MsgNull
 0001:D7FC       _SII68xMsgtxt
 0001:D804       _CMD64xMsgtxt
 0001:D80C       _PIIXxMsgtxt
 0001:D81A       _VIA571Msgtxt
 0001:D822       _SiS5513Msgtxt
 0001:D82A       _ALI5229Msgtxt
 0001:D832       _PDCxMsgtxt
 0001:D842       _ICHxMsgtxt
 0001:D84E       _HPT36xMsgtxt
 0001:D856       _AMDxMsgtxt
 0001:D85E       _AEC62xMsgtxt
 0001:D864       _OSBMsgtxt
 0001:D876       _NForceMsgtxt
 0001:D886       _ITEMsgtxt
 0001:D88E       _JMMsgtxt
 0001:D89C       _PromiseMIOtxt
 0001:D8AA       _MarvellMsgtxt
 0001:D8B6       _InitioMsgtxt
 0001:D8C6       _IDERMsgtxt
 0001:D8D6       _ParmErrMsg
 0001:D91A       _VersionMsg
 0001:D95E       _pcmdline1
 0001:D962       _pcmdline_slash
 0001:D966       _pcmdline_start
 0001:D96A       _tokv_index
 0001:D96C       _state_index
 0001:D96E       _length
 0001:D970       _tokvbuf
 0001:DA70       _pend_option
 0001:DA72       _ptable_option
 0001:DA74       _poutbuf1
 0001:DA76       _poutbuf_end
 0001:DA78       _cc
 0001:DA7C       _outbuf
 0001:DB7C       _outbuf_len
 0001:DB7E       _poutbuf
 0001:DB82       _OPT_NOTBEEP
 0001:DB8A       _OPT_NOT_BIOS
 0001:DB92       _OPT_NOT_BM_DMA
 0001:DB9A       _OPT_NOT_DM
 0001:DBA2       _OPT_NOTREMOVABLE
 0001:DBAA       _OPT_NOT_SETMAX
 0001:DBB2       _OPT_NOSHTDWN
 0001:DBBA       _OPT_NOT_SMS
 0001:DBC2       _OPT_NOT_VERBOSE
 0001:DBCA       _OPT_NOT_VPAUSE
 0001:DBD2       _OPT_80WIRE
 0001:DBDA       _OPT_ADAPTER
 0001:DBE2       _OPT_APM
 0001:DBEA       _OPT_BAY
 0001:DBF2       _OPT_BM_DMA
 0001:DBFA       _OPT_DEBUG
 0001:DC02       _OPT_DM
 0001:DC0A       _OPT_FIXES
 0001:DC12       _OPT_FORCEGBM
 0001:DC1A       _OPT_GBM
 0001:DC22       _OPT_IRQ
 0001:DC2A       _OPT_IDLETIMER
 0001:DC32       _OPT_IGNORE
 0001:DC3A       _OPT_LATENCY
 0001:DC42       _OPT_LOC
 0001:DC4A       _OPT_LPM
 0001:DC52       _OPT_MAXRATE
 0001:DC5A       _OPT_NOISE
 0001:DC62       _OPT_PCMCIA
 0001:DC6A       _OPT_PCICLOCK
 0001:DC72       _OPT_PORT
 0001:DC7A       _OPT_PF
 0001:DC82       _OPT_P
 0001:DC8A       _OPT_REMOVABLE
 0001:DC92       _OPT_SHTDWN
 0001:DC9A       _OPT_SMS
 0001:DCA2       _OPT_IRQTIMEOUT
 0001:DCAA       _OPT_T
 0001:DCB2       _OPT_UNIT
 0001:DCBA       _OPT_U
 0001:DCC2       _OPT_VERBOSE
 0001:DCCA       _OPT_VPAUSE
 0001:DCD2       _OPT_VERBOSEL
 0001:DCDA       _OPT_VPAUSEL
 0001:DCE2       _OPT_VERBOSELL
 0001:DCEA       _OPT_VPAUSELL
 0001:DCF2       _OPT_WP
 0001:DCFA       _OPT_END
 0001:DD02       _opttable
 0001:DD64       _DrvrNameTxt
 0001:DD72       _DrvrNameSize
 0001:DD74       _DrvrDescriptTxt
 0001:DD9A       _VendorNameTxt
 0001:DDA0       _DriverStruct
 0001:DDBC       _AdaptDescriptNameTxt
 0001:DDD2       _AdapterStruct
 0001:DDEA       _DevDescriptNameTxt
 0001:DDFA       _DevStruct
 0001:DE06       _VDMInt13Created
 0001:DE08       _VDMInt13Active
 0001:DE0A       _VDMInt13
 0001:DEBE       _VDMDskBlkID
 0001:DEC2       _VDMInt13BlkID
 0001:DEC6       _VPCIInfo
 0001:DEFE       _VPCardInfo
 0001:DF14       _VControllerInfo
 0001:DF46       _VUnitInfo1
 0001:DF62       _VUnitInfo2
 0001:DF84       _VModelInfo
 0001:DF90       _VModelUnknown
 0001:DF9C       _VBPBInfo
 0001:DFA2       _VI13Info
 0001:DFA8       _VIDEInfo
 0001:DFB2       _VGeomInfo0
 0001:DFF2       _VGeomInfo1
 0001:E022       _VGeomInfo2
 0001:E050       _VGeomInfo3
 0001:E086       _VBlankLine
 0001:E088       _VPauseVerbose0
 0001:E0B0       _VPauseVerbose1
 0001:E0D6       _VString
 0001:E0DA       _VSata0
 0001:E0E4       _VSata1
 0001:E0F0       _VSata2
 0001:E0FC       _VULTRADMAString
 0001:E10E       _VDMAString
 0001:E120       _VPIOString
 0001:E154       _counted
 0001:E4FA       _RMIDCTable
 0001:E550       _sbuf
 0001:E564       _fs
 0001:E576       _MemTop
 0001:E578       _Register
 0002:0008       _DSSel
 0002:000A       _CSSel
 0002:000C       _FlatSel
 0002:0010       ADD_InitTimer
 0002:0095       ADD_DeInstallTimer
 0002:00A9       ADD_StartTimerMS
 0002:011C       ADD_CancelTimer
 0002:013F       f_ADD_TimerHandler
 0002:0190       _APMAttach
 0002:01BE       _APMRegister
 0002:022B       _APMDeregister
 0002:0240       @safeXCHG
 0002:0243       @safeGET32
 0002:024C       @safeCLR32
 0002:0253       @safeDEC
 0002:025A       @safeINC
 0002:0261       @FixedIRQ0
 0002:0264       @FixedIRQ1
 0002:0267       @FixedIRQ2
 0002:026A       @FixedIRQ3
 0002:026D       @FixedIRQ4
 0002:0270       @FixedIRQ5
 0002:0273       @FixedIRQ6
 0002:0276       @FixedIRQ7
 0002:0278       @HandleInterrupts
 0002:02A0       _CSHookHandler
 0002:02BC       _LoadFlatGS
 0002:0328       @DevHelp_AllocGDTSelector
 0002:0346       @DevHelp_AttachDD
 0002:0360       @DevHelp_Beep
 0002:037A       @DevHelp_RegisterDeviceClassLite
 0002:03A6       @DevHelp_CreateInt13VDM
 0002:03C4       @DevHelp_SetIRQ
 0002:03DE       @DevHelp_UnSetIRQ
 0002:03F6       @DevHelp_EOI
 0002:040C       @DevHelp_GetDOSVar
 0002:0432       @DevHelp_Save_Message
 0002:044E       @DevHelp_VerifyAccess
 0002:0470       @DevHelp_VirtToPhys
 0002:049C       @DevHelp_PhysToVirt
 0002:04CC       @DevHelp_ProcRun
 0002:04EE       @DevHelp_ProcBlock
 0002:051A       @DevHelp_AllocateCtxHook
 0002:0542       @DevHelp_FreeCtxHook
 0002:055E       @DevHelp_ArmCtxHook
 0002:0588       @DevHelp_VirtToLin
 0002:05AC       @DevHelp_VMAllocLite
 0002:05DC       @DevHelp_LockLite
 0002:05F4       ADD_XFERIO
 0002:0874       @BuildSGList
 0002:0968       @OutB
 0002:0968       @OutB2
 0002:0994       @OutBdms
 0002:09A1       @OutBd
 0002:09B5       @OutW2
 0002:09B5       @OutW
 0002:09E1       @OutD2
 0002:09E1       @OutD
 0002:0A5D       @InB2
 0002:0A5D       @InB
 0002:0A89       @InBdms
 0002:0A8E       @InBd
 0002:0A99       @InW
 0002:0A99       @InW2
 0002:0AC5       @InWdms
 0002:0ACA       @InWd
 0002:0AD1       @InD2
 0002:0AD1       @InD
 0002:0B24       @InDdms
 0002:0B29       @InDd
 0002:0B32       _S506Str1
 0002:0EF2       @IssueCommand
 0002:0F46       @IssueCommandTO
 0002:0F66       @ClearIORB
 0002:0F8A       @DoSMART
 0002:1024       @GetSmartStatus
 0002:10C1       @IOCtlRead
 0002:1171       @GetInquiryData
 0002:1200       @IssueOneByte
 0002:1226       @IssueSetMax
 0002:1318       @IssueSetFeatures
 0002:1348       @IssueGetPowerStatus
 0002:1368       @IssueSetIdle
 0002:139D       @MapUnit
 0002:145B       @DoIOCTLs
 0002:1970       @StartSM
 0002:19FD       @FixedInterrupt
 0002:1A5C       @CatchInterrupt
 0002:1A87       @StartState
 0002:1B84       @StartIO
 0002:1BE4       @RetryState
 0002:1C1D       @InitACBRequest
 0002:1EB5       @SetupFromATA
 0002:2025       @SetupIdentify
 0002:20A5       @InitBlockIO
 0002:2125       @StartOtherIO
 0002:23C0       @StartBlockIO
 0002:2470       @SetIOAddress
 0002:25F0       @InterruptState
 0002:277F       @DoBlockIO
 0002:28B0       @DoOtherIO
 0002:2933       @DoneState
 0002:2B43       @ErrorState
 0002:2C9A       @SetRetryState
 0002:2D3F       @DoReset
 0002:2DDF       @ResetCheck
 0002:2F7C       @SendCmdPacket
 0002:2FEF       @WaitDRQ
 0002:3065       @CheckWorker
 0002:30D5       @CheckReady
 0002:30DD       @CheckBusy
 0002:30E5       @SelectUnit
 0002:3100       @SetMediaGeometry
 0002:3101       @GetChangeLine
 0002:311C       @GetLockStatus
 0002:3136       @GetUnitStatus
 0002:3168       @MapError
 0002:32AD       @MapMediaStatus
 0002:32D6       @CreateBMSGList
 0002:330C       _ADDEntryPoint
 0002:33BA       @NextIORB
 0002:3514       @FillUnitInfo
 0002:365F       @GetDeviceTable
 0002:38ED       @CompleteInit
 0002:3982       @AllocateUnit
 0002:399B       @DeallocateUnit
 0002:39B4       @ChangeUnitInfo
 0002:39F7       @GetQueueStatus
 0002:3A08       @GetUnitResources
 0002:3B9D       @Error
 0002:3BAD       @IORBDone
 0002:3BE2       @NotifyFLT
 0002:3C98       @Delay
 0002:3CAF       _APMEventHandler
 0002:3CEC       @InitUnitSync
 0002:3D55       @ReInitUnit
 0002:3D72       @UnitFlush
 0002:3D88       @APMSuspend
 0002:3DF7       @APMResume
 0002:3EE5       @ReConfigureUnit
 0002:3F50       @CardRemoval
 0002:3F93       @CardInsertion
 0002:3FAF       @StartDetect
 0002:4019       @IssueSATAReset
 0002:40ED       @SATARemoval
 0002:4129       @StartDetectSATA
 0002:4171       _InsertHandler
 0002:43E6       @CardInsertionDeferred
 0002:4504       _CSCallbackStub
 0002:451E       _IRQTimer
 0002:45FD       _DelayedRetry
 0002:461D       _DelayedReset
 0002:4638       _ElapsedTimer
 0002:4667       _IdleTicker
 0002:46BA       @IODly
 0002:46C5       @IODlyFar
 0002:46D0       @clrmem
 0002:46DD       @fclrmem
 0002:46F1       @strnswap
 0002:4738       @_strncmp
 0002:476A       @SuspendIORBReq
 0002:47F2       @Suspend
 0002:4813       @SuspendState
 0002:481A       @ResumeIORBReq
 0002:4845       @PreProcessIORBs
 0002:4970       @ReadConfigB
 0002:4998       @ReadConfigW
 0002:49BD       @ReadConfigD
 0002:49E6       @RConfigB
 0002:49F4       @RConfigW
 0002:4A00       @WriteConfigB
 0002:4A1B       @WriteConfigBI
 0002:4A32       @WriteConfigW
 0002:4A3D       @WriteConfigD
 0002:4A51       @WConfigBI
 0002:4A5D       @WConfigB
 0002:4A6B       @WConfigW
 0002:4A77       @WConfigD
 0002:4A90       __aNlshl
 0002:4A9B       __aFlshl
 0002:4AA6       __aNulshr
 0002:4AB1       __aFulshr
 0002:4ABC       __aNulmul
 0002:4ABC       __aNlmul
 0002:4AD0       __aNNalmul
 0002:4AD0       __aNNaulmul
 0002:4AE9       __aFulmul
 0002:4AE9       __aFlmul
 0002:4AFD       __aNuldiv
 0002:4B14       __aFuldiv
 0002:4B2B       __aNulrem
 0002:4B44       __aFulrem
 0002:4B5D       _CalculateLoss
 0002:4B80       _MPIfIOCtl
 0002:4C7E       @FindAdapterForSocket
 0002:4CB3       _CSCallbackHandler
 0002:4D7C       @DoIOCtlPCMCIA
 0002:4E32       __aNFaulshr
 0002:4E50       __aNFauldiv
 0002:4E76       __aNFaulrem
 0002:4E9C       _NotifyIORBDone
 0002:4EC2       @TestStatus50us
 0002:4EF8       @WaitNotBusy
 0002:4F4B       @WaitNotBusyDRQ
 0002:4F98       @TryCommand
 0002:4FEF       @TestChannel
 0002:529E       @CheckController
 0002:531E       @Execute
 0002:5379       @NoOp
 0002:53BE       @HookIRQ
 0002:543B       @UnhookIRQ
 0002:545C       @RehookIRQ
 0002:5486       @DriveInit
 0002:57C5       @SetupPCMCIA
 0002:580D       @SetupPCI
 0002:584D       @AssignPCIChips
 0002:585E       @NoMaster
 0002:5881       @AddUnit
 0002:58C0       @ScanForUnits
 0002:597F       @AssignSGList
 0002:5A17       @VerifyInitPost
 0002:5ACC       @ConfigureACB
 0002:5C6D       @ConfigurePCCard
 0002:5D08       @CollectPorts
 0002:5D94       @ConfigureController
 0002:5FEE       @ConfigureUnit
 0002:608E       @ReadDrive
 0002:6156       @TraceCh
 0002:6168       _TraceStr
 0002:6194       @TraceTime
 0002:61C6       @TraceTTime
 0002:6206       @DiffTime
 0002:6223       @TotalTime
 0002:6240       @TWrite
 0002:6271       @RegisterADD
 0002:6289       @UCBSetupDMAPIO
 0002:636B       @CountBits
 0002:6387       @GetDeviceULTRAMode
 0002:6498       @GetDeviceDMAMode
 0002:6565       @GetDevicePIOMode
 0002:65F1       @GetChipPIOMode
 0002:6674       @IdentifyDevice
 0002:6826       _sprntf
 0002:683A       @prntf
 0002:6CA6       @_strncpy
 0002:6D04       @DetermineUnitGeometry
 0002:6EF0       @AdjustCylinders
 0002:6F69       @IdentifyGeometryGet
 0002:701A       @UnlockMax
 0002:7249       @IDEGeomExtract
 0002:7394       @LogGeomCalculate
 0002:7400       @LogGeomCalculateLBAAssist
 0002:74CC       @Int13GeometryGet
 0002:7592       @CheckLVM
 0002:75E1       @CheckMBRConsistency
 0002:7727       @BPBGeometryGet
 0002:7AC6       @ReadAndExtractBPB
 0002:7B17       @PhysGeomValidate
 0002:7B34       @IDStringsExtract
 0002:7B71       @MediaStatusEnable
 0002:7BF6       @MultipleModeEnable
 0002:7C9A       @IdleTimerEnable
 0002:7D23       @AcousticEnable
 0002:7D7D       @APMEnable
 0002:7D9C       @LPMEnable
 0002:7E0E       @SetupCommonPre
 0002:80A4       @SetupCommonPost
 0002:81F6       @SetupCommon
 0002:8232       @PickClockIndex
 0002:8297       @CalculateAdapterTiming
 0002:82F4       @GetPIIXPio
 0002:8373       @GetSCHPio
 0002:8398       @PIIXTimingValue
 0002:843B       @ProgramPIIXChip
 0002:85DA       @ProgramSCH
 0002:8658       @GetVIAPio
 0002:8692       @VIATimingValue
 0002:874E       @ProgramVIAChip
 0002:8892       @GetNetCellPio
 0002:88B1       @GetGenericPio
 0002:88D3       @CalculateGenericAdapterTiming
 0002:895D       @NonsharedCheckIRQ
 0002:8A11       @BMCheckIRQ
 0002:8A91       @GenericSetTF
 0002:8B8E       @GenericGetTF
 0002:8C74       @GenericStartOp
 0002:8CB7       @GenericSetupDMA
 0002:8CE5       @GenericStopDMA
 0002:8D0C       @GenericErrorDMA
 0002:8D20       @GetALIPio
 0002:8D54       @SetupALI
 0002:8DA3       @ALITimingValue
 0002:8E47       @ProgramALIChip
 0002:8F0E       @GetSISPio
 0002:8F5A       @SISTimingValue
 0002:8FEA       @SIS2TimingValue
 0002:904B       @ProgramSISChip
 0002:9092       @ProgramSIS2Chip
 0002:90CC       @GetCMDPio
 0002:912D       @CMDTimingValue
 0002:91D3       @ProgramCMDChip
 0002:9313       @CMDCheckIRQ
 0002:9390       @GetPDCPio
 0002:93AF       @SetupPDCTX2
 0002:93CE       @PDCTimingValue
 0002:94B3       @ProgramPDCIO
 0002:9562       @ProgramPDCChip
 0002:96A2       @ProgramPDCChipTX2
 0002:96B9       @PromiseTX2CheckIRQ
 0002:9749       @PromiseCheckIRQ
 0002:981E       @PDCPostReset
 0002:9841       @PDCPreReset
 0002:9856       @PDCSetupDMA
 0002:98A6       @PDCStartOp
 0002:990F       @PromiseMSetupDMA
 0002:9923       @PromiseMStartOp
 0002:99A1       @PromiseMStopDMA
 0002:99D4       @PromiseMErrorDMA
 0002:99D5       @PromiseMCheckIRQ
 0002:9A7E       @GetCxPio
 0002:9AB6       @CxTimingValue
 0002:9B4D       @ProgramCxChip
 0002:9BB2       @HPTClkIdx
 0002:9BFF       @GetHPTPio
 0002:9C3D       @HPTTimingValue
 0002:9CD7       @ProgramHPTChip
 0002:9D8A       @HPTCheckIRQ
 0002:9DF9       @HPTEnableInt
 0002:9E08       @HPT36xPreReset
 0002:9E13       @HPT37xPreReset
 0002:9E30       @HPT36xSetupDMA
 0002:9E5A       @HPT37xSetupDMA
 0002:9E8D       @HPT36xErrorDMA
 0002:9EA9       @HPT37xErrorDMA
 0002:9ECA       @GetAECPio
 0002:9F1A       @AECTimingValue
 0002:9F8D       @ProgramAECChip
 0002:A036       @GetAEC2Pio
 0002:A04E       @AEC2TimingValue
 0002:A08F       @ProgramAEC2Chip
 0002:A0A8       @GetOSBPio
 0002:A0D4       @OSBTimingValue
 0002:A163       @ProgramOSBChip
 0002:A268       @ReadIDEReg
 0002:A29A       @GetOPTIPio
 0002:A2D1       @OPTITimingValue
 0002:A373       @ProgramOPTIChip
 0002:A48A       @GetSIIPio
 0002:A4B1       @GetSIISATAPio
 0002:A4EE       @SIITimingValue
 0002:A59C       @ProgramSIIChip
 0002:A618       @ProgramSIISATAChip
 0002:A654       @SIISetTF
 0002:A689       @SIIStartOp
 0002:A71A       @SIIStartStop
 0002:A79D       @SIICheckIRQ
 0002:A854       @ITETimingValue
 0002:A8D1       @ProgramITEChip
 0002:A926       @GetJMBPio
 0002:A948       @InitioSetupDMA
 0002:A95C       @InitioStartOp
 0002:A995       @InitioStopDMA
 0002:A9B5       @InitioErrorDMA
 0002:A9B6       @InitioCheckIRQ
 0002:AA48       __CodeEnd
 0003:0000       _CallCardServices
 0003:004A       @PCMCIASetup
 0003:007C       @CardServicesPresent
 0003:0108       @CSCardPresent
 0003:029A       @CSRegisterClient
 0003:02E9       @CallCS
 0003:0345       @TryIRQ
 0003:0382       @TryIO
 0003:03A2       @CSConfigure
 0003:0800       @CSReconfigure
 0003:083E       @CSUnconfigure
 0003:08DC       @ACPISetup
 0003:090B       @ACPIGetPCIIRQs
 0003:096C       _StubVDMInt13CallBack
 0003:0973       @CallOEMHlp
 0003:09AA       @CallAcpiCA
 0003:09E6       @PciSetReg
 0003:0A38       @PciGetReg
 0003:0A94       @SetRegB
 0003:0AAA       @SetRegW
 0003:0AB4       @SetRegD
 0003:0AC7       @GetRegB
 0003:0AED       @GetRegW
 0003:0B11       @GetRegD
 0003:0B39       @ReadPCIConfigSpace
 0003:0C99       @WritePCIConfigSpace
 0003:0DEE       @ConfigurePCI
 0003:0FCE       @ScanForOtherADDs
 0003:1091       @SetOption
 0003:10DB       @ParseCmdLine
 0003:1501       @PortToPhys
 0003:155A       @PrintAdapterInfo
 0003:16BD       @PrintInfo
 0003:1A1D       @SaveMsg
 0003:1A85       @TTYWrite
 0003:1ABB       @ProcessVerboseTimings
 0003:1B6F       @AllocResource
 0003:1BFB       @AllocAdapterResources
 0003:1D1E       @DeallocAdapterResources
 0003:1D59       @AssignAdapterResources
 0003:1EAD       @FindHotPCCard
 0003:1F96       @LocateATEntry
 0003:2006       @Command_Parser
 0003:274C       @SetupOEMHlp
 0003:27D3       @GetPCIBuses
 0003:27ED       @CheckLegacyPorts
 0003:2859       @SetLatency
 0003:28AF       @CheckWellknown
 0003:2945       @GetBAR
 0003:2A46       @ProbeChannel
 0003:2B96       @SetupT13StandardController
 0003:2C3B       @CheckSATAPhy
 0003:2CC6       @CollectSCRPorts
 0003:2D20       @nextController
 0003:2E6E       @EnumPCIDevices
 0003:3251       @HandleFoundAdapter
 0003:339A       @VDMInt13Create
 0003:343D       @Int13Fun08GetLogicalGeom
 0003:349A       @Int13DoRequest
 0003:34DC       _VDMInt13CallBack
 0003:3512       @AcceptPIIX
 0003:386E       @AcceptSCH
 0003:38AB       @AcceptSMSC
 0003:38DB       @AcceptITE8213
 0003:3924       @AcceptVIA
 0003:3D48       @AcceptAMD
 0003:3E1D       @AcceptNVidia
 0003:4016       @AcceptGeneric
 0003:40A6       @AcceptNetCell
 0003:40BB       @AcceptMarvell
 0003:4166       @AcceptAHCI
 0003:4216       @GenericInitComplete
 0003:4217       @GenericSATA
 0003:4230       @GetAHCISCR
 0003:42B6       @AcceptALI
 0003:45F4       @AcceptSIS
 0003:49AE       @AcceptCMD
 0003:4AB0       @AcceptPDC
 0003:4B3E       @AcceptPDCTX2
 0003:4B9D       @PromiseInitComplete
 0003:4C17       @AcceptPDCMIO
 0003:4F12       @AcceptCx
 0003:4F26       @SetupHPTPLL
 0003:504E       @AcceptHPT
 0003:51BE       @AcceptAEC
 0003:5238       @AcceptAEC2
 0003:52C2       @AcceptOSB
 0003:537D       @AcceptIXP
 0003:53CC       @AcceptBCM
 0003:5442       @AcceptOPTI
 0003:5488       @SiISATA
 0003:5652       @AcceptSII
 0003:56C9       @AcceptIXPSATA
 0003:56DA       @AcceptITE
 0003:57A0       @AcceptJMB
 0003:5908       @AcceptInitio
 0003:5AD0       MY_DEVHELP_ATTACHDD
 0003:5AF2       _RMCreateDriver
 0003:5B6C       _RMDestroyDriver
 0003:5B98       _RMCreateAdapter
 0003:5BD2       _RMCreateDevice
 0003:5C0C       _RMAllocResource
 0003:5C46       _RMDeallocResource
 0003:5C72       _CallRM
 0003:5C9A       _GetCS
 0004:0000       _MsgBuffer
 0004:FFFF       _MsgBufferEnd
